:020000040007F3
:10800000E0580020D9830700E1830700E3830700DD
:10801000E5830700E7830700E9830700000000000D
:10802000000000000000000000000000C583070001
:10803000ED83070000000000EF830700F1830700D5
:10804000F3830700F3830700F3830700F38307003C
:10805000F3830700F3830700F3830700F38307002C
:10806000F3830700F3830700F3830700F38307001C
:10807000F3830700F3830700F3830700F38307000C
:1080800031960700F3830700F3830700F3830700AB
:10809000F3830700F3830700A1940700F38307002D
:1080A000F3830700F3830700F3830700F3830700DC
:1080B000F3830700F38307000000000000000000C6
:1080C000F3830700F3830700F3830700F3830700BC
:1080D0002D940700F3830700F3830700F383070061
:1080E000F383070000000000000000000000000013
:1080F00000000000F383070000000000F383070086
:10810000000000000000000000000000000000006F
:10811000000000000000000000000000000000005F
:10812000000000000000000000000000000000004F
:10813000000000000000000000000000000000003F
:10814000000000000000000000000000000000002F
:10815000000000000000000000000000000000001F
:10816000000000000000000000000000000000000F
:1081700000000000000000000000000000000000FF
:1081800000000000000000000000000000000000EF
:1081900000000000000000000000000000000000DF
:1081A00000000000000000000000000000000000CF
:1081B00000000000000000000000000000000000BF
:1081C00000000000000000000000000000000000AF
:1081D000000000000000000000000000000000009F
:1081E000000000000000000000000000000000008F
:1081F000000000000000000000000000000000007F
:10820000DFF810D000F03AF90048004741A6070017
:10821000AFF30080E058002030B450E8012F93B253
:10822000C48923448489A34228BF1B1B0489A34219
:1082300002BFBFF32F8F002007E0C3EA020340E82C
:108240000134002CE9D14FF001000A6030BC7047C6
:1082500050E8012FC2EA024240E801210029F7D18B
:10826000704730B450E8022F1FFAA2F3C488A3422B
:1082700002BFBFF32F8F00200DE0C48923448489FF
:10828000A34228BF1B1BC2EA034340E80234002C70
:10829000E8D14FF001000A6030BC704750E8022F6F
:1082A000C2EA224240E802210029F7D17047034682
:1082B00053E8022FD988B2EB324F4FF0000017BFBE
:1082C00092B241EA014142EA014104E05A68B2EB4C
:1082D000324F08BF012043E80212002AE8D170475C
:1082E00030B4044654E8000F0D4644E80053002B18
:1082F000F8D1156030BC704730B4044654E8000F24
:1083000040EA010544E80053002BF7D1156030BC6A
:10831000704730B4044654E8000F00EA010544E811
:108320000053002BF7D1156030BC704730B40446C1
:1083300054E8000F80EA010544E80053002BF7D110
:10834000156030BC704730B4044654E8000F00EBB1
:10835000010544E80053002BF7D1156030BC70478D
:1083600030B4044654E8000FA0EB010544E8005384
:10837000002BF7D1156030BC704770B404464FF045
:10838000000054E8006F0D68AE4207BF44E80023C8
:10839000012044E800630E60002B1CBF0020F0E7C2
:1083A00070BC704730B4044654E8000F88422CBFBC
:1083B000451A054644E80053002BF5D1156030BC42
:1083C000704700001EF0040F0CBFEFF30880EFF3BE
:1083D000098003F071BC000006488047064800474A
:1083E000FEE7FEE7FEE7FEE7FEE7FEE7FEE7FEE765
:1083F000FEE7FEE7A594070001820700202A04DBC0
:10840000203A00FA02F1002070479140C2F12003A7
:1084100020FA03F319439040704740EA01039B0799
:1084200003D009E008C9121F08C0042AFAD203E0E9
:1084300011F8013B00F8013B521EF9D27047D2B24D
:1084400001E000F8012B491EFBD270470022F6E73D
:1084500010B513460A4604461946FFF7F0FF2046BA
:1084600010BD30B504460020034600E05B1C93427B
:1084700003D2E05CCD5C401BF8D030BD064C074D0C
:1084800006E0E06840F0010394E8070098471034E4
:10849000AC42F6D3FFF7B8FEACDA0700CCDA07003F
:1084A0002DE9F0438BB01446129D15F9046B00962C
:1084B0001F46804689462B460246214602A800F008
:1084C00084FC02A9129A084600F07BFC129B02AAC7
:1084D0004146404600F065FC129B02AA2146204618
:1084E00000F05FFC2B464A4639463846009600F0BD
:1084F0006CFC129A394602A800F063FC02A92B46D4
:1085000042460846009600F060FC02A92B4622462F
:108510000846009600F059FC2B464246214620466C
:10852000009600F052FC129B22464946484600F055
:1085300038FC2B4602AA41462046009600F045FC36
:10854000129B22463946384600F02BFC2B464A4601
:1085500039463846009600F038FC324602A92046DB
:1085600000F0FAFD0BB0BDE8F083F0B5154689B018
:108570001C4607460E461A462946684600F021FC6E
:1085800023466A463946384600F00BFC23462A4605
:108590006946684600F005FC23466A463146304687
:1085A00000F0FFFB09B0F0BD8B1802448B4200D1F4
:1085B000704713F8010D02F8010DF7E72DE9F047B8
:1085C000B3F9024088461E4604F11F0120230734F8
:1085D00091FBF3F708234FFA87F994FBF3F49442E5
:1085E00028BF14464946054600F070FA2246414627
:1085F000FFF7DAFFB6F90230E4009C421FD9E41A13
:1086000005EB87010022C4F120078D420ED32436EA
:108610004A462946304600F064FA01280FD04B46FE
:1086200032462846BDE8F04700F0A2BD51F8040DDF
:1086300020FA04F313430B6000FA07F2E5E7BDE804
:10864000F0872DE9F04793F9006092B0044689461F
:10865000104631461546984600F058FA002840F07A
:1086600091804246494602A800F0ABFB434602AA6D
:1086700021460AA800F095FB02A90846424600F0F0
:10868000A0FB43462A464946484600F08AFB08F1CB
:10869000040742462946284600F093FB3B462A46FB
:1086A00021462046009600F040FA3B462A462946DD
:1086B0002846009600F039FA3B462A4621462846CD
:1086C000009600F082FB43462A462146204600F0F1
:1086D00068FB3B46224621462846009600F025FAD4
:1086E0003B4600962A462146204600F01EFA2368A3
:1086F000DB074AD533463A462146204600F0B8F912
:1087000031468246204600F01AFD06F18043013BC7
:1087100054F8230040EACA7044F823004246214638
:10872000284600F04EFB3B460AAA294628460096FA
:1087300000F04BFB3B460AAA29462846009600F06B
:1087400044FB0AA908463B462A46009600F03DFB3A
:1087500043460AAA2146204600F023FB02AA3B46D4
:1087600010462146009600F030FB3246294620464E
:1087700000F0F2FC4946284600F0EEFC02A948460B
:1087800000F0EAFC12B0BDE8F0873146204600F068
:10879000D6FCC3E700487047FCD907002DE9F04F2D
:1087A000EDB01F46DDF8D8810590B8F9026098F960
:1087B000004020231F3696FBF3F676B206F1FF3910
:1087C00024AB002543F829506CAB03EB89034CA87C
:1087D0008A469346394698F9012043F8805C43F86D
:1087E000605CFFF7E1FE98F9012054A8B918FFF783
:1087F000DBFE21464CA800F089F90746002840F02E
:108800002E8154A800F082F90290002840F02981BE
:1088100008F1240332464CA91846039300F061F98D
:10882000012840F02081324654A9039800F059F9FC
:108830000128069040F017811CAD0CAF3346039A17
:1088400054A9284600F08AF9029B47F829305A4675
:10885000514638464346FFF7B1FE39463846039B3A
:1088600000962A4600F0FDF90DF5B879039B0096B5
:108870002A464CA914A800F0F4F922464846059966
:1088800000F06AFCA30009EB030A0793059BA10013
:10889000591808F1440B504600F05EFC594634A8C4
:1088A00000F05AFCA3000BEB03013CA800F054FCC1
:1088B00008F10403494634AA28460094049300F0C2
:1088C00084FA53464A463CA934A8CDF80080FFF705
:1088D000E7FD2346049A2946284600F03FF92A4638
:1088E000514648464346FFF740FE029BCDE9083B10
:1088F000059B31463846CDE90A3900F001FC314686
:10890000814614A800F0FCFB8145B8BF81461FFAE0
:1089100089F909F1FF3B0FFA8BFB5946384600F005
:1089200057FC5946071C14A818BF012700F050FC3B
:10893000002814BF022300231F430DF1200A224602
:108940005AF8277024A8394600F006FC0DF1B00B48
:10895000A300F918584600F0FFFB2146284600F016
:10896000B5F8A9F10209069B2B600FFA89F90DF100
:10897000900AB9F1000F23DA2346049A29462846C3
:1089800000F0ECF843462A4659465046FFF7EDFD05
:1089900032465146039800F0A4F8012804D033462B
:1089A000039A504600F0E4FB013C64B24CAA230653
:1089B0004BD5029BB3FA83F040096DB0BDE8F08F50
:1089C00043462A46D8F8A47059465046B847494607
:1089D0000CA800F0FDFB4946071C14A818BF01278E
:1089E00000F0F6FB002814BF022300231F4308AB4E
:1089F00053F8277027B32246394634A800F0ACFB61
:108A0000079B3CA8F91800F0A7FB43462A463CA95F
:108A100034A8FFF7AAFD049B009434AA514644A849
:108A200000F0D3F95B4652463CA934A8CDF800804B
:108A3000FFF736FD434644AA2946284600F0B1F91F
:108A400009F1FF390FFA89F993E752F824105AF81F
:108A500024304B40029919430291013CA7E7284674
:108A6000ABE73846A9E70298A7E70000000000003E
:108A7000C3F10803DB0070B50133002403A500BF78
:108A80005B1920C940CAAD1920C0184720C940CA87
:108A9000754120C020C940CA754120C020C940CAC4
:108AA000754120C020C940CA754120C020C940CAB4
:108AB000754120C020C940CA754120C020C940CAA4
:108AC000754120C06441204670BD00BF002310B531
:108AD0001C465AB2914200DC10BD40F823400133DD
:108AE000F7E710B5013A52B2130601D5002010BDC8
:108AF00050F8224051F822309C4205D802F1FF3252
:108B0000F2D24FF0FF30F2E70120F0E710B500237A
:108B10001A465CB2A14203DCB2FA82F0400910BDF1
:108B200050F8234001332243F3E770B59DF910401C
:108B30001E4623460546FFF79BFF30B922462946CD
:108B40003046FFF7CEFF012807D02346324629469C
:108B50002846BDE8704000F00BBB70BDF0B50F4675
:108B6000A1B006461946384615461C46FFF7CEFF0B
:108B700020B13046FFF7AAFF21B0F0BD22463946AA
:108B8000684600F0E9FA294608A800F0E5FA10A8BE
:108B90002146FFF79BFF012318A81093FFF796FFCC
:108BA000224608A96846FFF79CFF28B9224610A96B
:108BB000304600F0D1FADFE7009BDA0709D42146FE
:108BC000684600F0BCFA2246294610A800F0E0FBF7
:108BD000E6E7089BDB0707D4214608A800F0AFFAB8
:108BE0002246294618A8F1E7002823461CDD08AADA
:108BF0006946684600F0BCFA2146684600F09FFAD4
:108C0000224618A910A8FFF76CFF002805DA10A962
:108C100023462A460846FFF72BFF10A9234618AA29
:108C2000084600F0A5FACEE708A96A46084600F013
:108C30009FFA214608A800F082FA224610A918A837
:108C4000FFF74FFF002805DA18A923462A460846F1
:108C5000FFF70EFF18A9234610AA084600F088FA6D
:108C6000BEE72DE9F04FB5B004AD9DF9F8401F46C1
:108C700081462346284600F0BAF824AB2146384600
:108C8000CDE9023500F03CFAC0EB841005B26B422E
:108C900003F01F034FF0200695FBF6F676B205F0C1
:108CA0001F0814A858BFC3F100083146FFF70EFF94
:108CB000B8F1000F30B22DDD14AB002203EB8000C1
:108CC000C8F1200C1346A34219D327B27B000193AD
:108CD00014AB03EB870704F1FF3834AB012603EB39
:108CE0008808002D53DA34AB03EB8606224656F88B
:108CF000C81C484600F030FA35B0BDE8F08F57F890
:108D0000236006FA08F10A4340F8232026FA0CF201
:108D10000133D8E714AB2246394603EB800000F05C
:108D20001BFAD2E70FFA82FE5AF8C83C53F82EB06D
:108D300034AB03EB820252F8803CABEB03031B1A0B
:108D40009B4502D034BF012000205CF8C82C42F8BB
:108D50002E300131019B4AB29A42E3DB331A5E4264
:108D6000214614A85E4100F0EAF934AB03EB84031A
:108D7000214653F8802C58F8803C384643EAC273A9
:108D8000013D48F8803C2DB200F0D9F9A9E734AB99
:108D90000021C6F1010C084603EB860A03EB8C0C9C
:108DA000D8E730B51C4691B0054693F900306846C7
:108DB00000F01DF8D4F8AC3069462846984711B049
:108DC00030BD13460A46FFF7ECBF70B59DF9104061
:108DD0001E462346054600F0CBF938B123463246FD
:108DE00029462846BDE87040FFF742BE70BD2DE918
:108DF000F04F08B4F8CA04B451F8042BA3FB02895D
:108E000040F8048B4FF0000AE4FB629A4FF0000B2D
:108E1000E5FB62AB4FF0000CE6FB62BC4FF0000ECE
:108E2000E7FB62CE51F8042B4FF00008E3FB6289A8
:108E300040F8048BE4FB629AE5FB62ABE6FB62BCA4
:108E4000E7FB62CE51F8042B4FF00008E3FB628988
:108E500040F8048BE4FB629AE5FB62ABE6FB62BC84
:108E6000E7FB62CE51F8042B4FF00008E3FB628968
:108E700040F8048BE4FB629AE5FB62ABE6FB62BC64
:108E8000E7FB62CE51F8042B4FF00008E3FB628948
:108E900040F8048BE4FB629AE5FB62ABE6FB62BC44
:108EA000E7FB62CE40F8049B40F804AB40F804BBFB
:108EB00040F804CB40F804EB0CBC052B00F01E81FD
:108EC0000C68A0F11400A1F11401A2F1140252F8EF
:108ED00004EB4FF0000550F8046BE4FB6E5652F8BB
:108EE00004EB50F8047BE4FB6E6752F804EB50F897
:108EF000048BE4FB6E7852F804EB50F8049BE4FB1F
:108F00006E8952F804EB50F804ABE4FB6E9AA0F1C2
:108F1000140052F8044B51F804EB4FF0000CE4FB42
:108F20006EC540F804CB51F804EBE4FB6E5640F8F4
:108F3000045B51F804EBE4FB6E6740F8046B51F8F6
:108F400004EBE4FB6E7840F8047B51F804EBE4FB9F
:108F50006E8940F8048B51F804EBE4FB6E9AA0E8AC
:108F60000006062B00F0CA800C68A0F11800A1F1E1
:108F70001801A2F1180252F804EB4FF0000550F866
:108F8000046BE4FB6E5652F804EB50F8047BE4FBF0
:108F90006E6752F804EB50F8048BE4FB6E7852F8DD
:108FA00004EB50F8049BE4FB6E8952F804EB50F894
:108FB00004ABE4FB6E9A52F804EB50F804BBE4FBFC
:108FC0006EABA0F1180052F8044B51F804EB4FF0CF
:108FD000000CE4FB6EC540F804CB51F804EBE4FB55
:108FE0006E5640F8045B51F804EBE4FB6E6740F802
:108FF000046B51F804EBE4FB6E7840F8047B51F805
:1090000004EBE4FB6E8940F8048B51F804EBE4FBBD
:109010006E9A40F8049B51F804EBE4FB6EABA0E8B9
:10902000000C072B6AD008B40C68A0F11C00A1F159
:109030001C01A2F11C0252F804EB4FF0000550F89D
:10904000046BE4FB6E5652F804EB50F8047BE4FB2F
:109050006E6752F804EB50F8048BE4FB6E7852F81C
:1090600004EB50F8049BE4FB6E8952F804EB50F8D3
:1090700004ABE4FB6E9A52F804EB50F804BBE4FB3B
:109080006EAB52F804EB50F804CBE4FB6EBCA0F1DD
:109090001C0052F8044B51F804EB4FF00003E4FBC2
:1090A0006E3540F8043B51F804EBE4FB6E5640F893
:1090B000045B51F804EBE4FB6E6740F8046B51F875
:1090C00004EBE4FB6E7840F8047B51F804EBE4FB1E
:1090D0006E8940F8048B51F804EBE4FB6E9A40F87B
:1090E000049B51F804EBE4FB6EAB40F804AB51F881
:1090F00004EBE4FB6EBCA0E8001808BCBDE8F08FF0
:10910000013949B20A06CBB205D4013900EB81021C
:109110005268002AF6D001335BB273B103F180428A
:10912000013A50F82220002022B9013B00EB431302
:1091300018B2704752080130F6E71846704700EB46
:1091400081010023884200D3704751F8042D43EA7F
:1091500052030B60D307F5E710B500235CB2A242BF
:1091600000DC10BD51F8234040F823400133F5E7FF
:10917000C3F10803DB0070B50133002403A500BF71
:109180005B1920C940CAAD1B20C0184720C940CA7E
:10919000B54120C020C940CAB54120C020C940CA3D
:1091A000B54120C020C940CAB54120C020C940CA2D
:1091B000B54120C020C940CAB54120C020C940CA1D
:1091C000B54120C06441B4FA84F0400970BD00BFCD
:1091D0004A11012350F8220001F01F0103FA01F1A6
:1091E00008407047F0B5082289B00C460646FFF7E4
:1091F000B3FFCB6A03930B6B04934B6B05938B6BA1
:109200000693CB6B0793002708236A466946684696
:10921000CDE901770097FFF72BFC082305466A4646
:1092200031463046FFF724FC236B0393636B0493B2
:10923000A36B0593E36B0544CDE906376A46082323
:1092400069466846FFF714FC082305446A46314620
:109250003046FFF70DFC236A0093636A0193A36A0B
:109260000293A36B0693E36B0793054408236A46B6
:1092700031463046CDE904770397FFF7F9FB636A7F
:109280000093A36AA26B0193E36A02930492636B57
:10929000E26B0393CDE90523236A07930544082372
:1092A0006A4631463046FFF7E3FBE36A0093236BDF
:1092B0000193636B0293236A0693A36A07930544A1
:1092C00008236A4631463046CDE904770397FFF715
:1092D0004FFF236B0093636B0193A36B0293E36BCC
:1092E0000393636A0693E36A07932D1A08236A4679
:1092F00031463046CDE90477FFF73AFF636B0093C0
:10930000A36B0193E36B0293236A0393636A049351
:10931000A36ACDE90537236B07932D1A08236A4604
:1093200031463046FFF724FFA36B0093E36BCDE992
:109330000137636A0393A36A0493E36ACDE90537AF
:10934000636B07932D1A08236A4631463046FFF7B0
:109350000FFF2D1A0D4C0FD435B908223146204687
:10936000FFF7BFFB01280FD00823224631463046C5
:10937000FFF7FEFE2D1AEFE708232246314630465E
:10938000FFF776FB2D18F7D409B0F0BD00DA07001F
:1093900070B5036813F001050646144605D0134660
:1093A0000A460146FFF764FB054621463046FFF7B3
:1093B000C6FE45B104F18042013A56F8223043F02E
:1093C000004346F8223070BD2DE9F0438BB00446CF
:1093D000154689460AAE1C22002103A8FFF738F87B
:1093E000032346F8203D95F900802A464946204649
:1093F0002F1DFFF7E6FC3B46324621462046CDF8BE
:109400000080FFF7E2FC2B464A4621462046FFF744
:10941000C8FCCDF800803B4605F184022146204679
:10942000FFF783FB0BB0BDE8F08300002DE9F041AE
:10943000194E4FF48271D6F8040130B11748C26852
:10944000521CC260304602F0CFFA00254FF4A077DC
:1094500007EB85018AB23046B258BAB189B202F040
:10946000C3FA0E48103000EB0514204603F01EFF2F
:10947000616819B1204603F0A1FE07E0A16811B1AF
:10948000204603F09BFE206800B180476D1C022D32
:10949000DED3BDE8F081000000400240F42A002045
:1094A00002F09EBB10B54FF080520023D2E94C1061
:1094B0000D2906D18C07C4F80C31C4F81031534C77
:1094C00023600D2955D1524B1B68524C2360504BE1
:1094D0001B1D1B68241D23604D4B08331B68241D76
:1094E00023604B4B0C331B68241D2360484B103307
:1094F0001B68241D2360464B14331B68241D236006
:10950000434B18331B68434C20342360404B1C33BF
:109510001B68241D23603E4B20331B68241D2360E1
:109520003B4B24331B68241D2360394B28331B68B5
:10953000241D2360364B2C331B68241D2360344BC1
:1095400030331B68334C40342360314B34331B6859
:10955000241D23602E4B38331B68241D23602C4BA5
:109560003C331B68241D2360294B40331B68241D9A
:1095700023600D2906D128480168C90702D06FF081
:10958000010101602548016841F470010160BFF3E9
:109590004F8FBFF36F8FD2E94C104FF010220D297F
:1095A00007D130B1012804D0D2F808021749203180
:1095B0000860D2F80002002803DBD2F80402002879
:1095C0001FDA012002F0C6FB1221C2F80012144873
:1095D0000368002BFCD0C2F8041201680029FCD0FB
:1095E000002002F0B7FBBFF34F8F0C487C380168B6
:1095F0000C4A01F4E06111430160BFF34F8F00BFDB
:10960000FDE70A490848086010BD00003805004021
:109610000404001020C500400004004088ED00E074
:1096200000E401400400FA050090D0038C2B0020D8
:10963000034808B5002101600068009008BD0000E3
:109640000001014002E008C8121F08C1002AFAD137
:1096500070477047002001E001C1121F002AFBD1B2
:10966000704700000121202803DA814005480140AD
:1096700003E0402802DA2038814009B10120704718
:1096800000207047FC06FFBD800701D00020704716
:1096900001207047C3688B4206D811440069491EF7
:1096A000814201D8012070470020704730B585B055
:1096B0000D46164C1621ADF800101ECC0DF1040C11
:1096C0008CE81E00124C0221012221706270A070F1
:1096D0000320E070217159206071FE20A07169465D
:1096E00004F109007DDF00280ED1BDF800002A46F4
:1096F000411CE17109212172BDF808100844ADF840
:10970000080001A9034872DF05B030BDB0D60700DC
:10971000C42F00202C2B002010B586B00624182260
:1097200008496846FEF779FE69462046FFF7BEFF06
:10973000002805D1044C207874DF0121207873DFE4
:1097400006B010BDC0D607002C2B002070B5104C01
:10975000A66C656A01F0ECFA216B08446A1A314480
:10976000814200D10022082300F0A4FE06000DD1A2
:1097700001F0DEFA0022294600F0EAFBA16A8142EC
:1097800003D10121A561C4E90701304670BD000085
:109790005C47002002F0E0FB02F0DEFB2DE9F84F11
:1097A000254C8146924660880E46814241D800276A
:1097B0004FF6FF788DF80070684600F075F8227853
:1097C0006078A188884201DA401C00E00020C0B225
:1097D000904204D19DF8000000F08AF827E06578F7
:1097E0006078884201DA401C00E0002060709DF83B
:1097F000000000F07DF8454519D0A068B9F1000FD0
:1098000040F835A00DD066B16188E068324605FBAE
:1098100001004946FEF701FEA06800EBC500868006
:1098200002E000EBC50087800020BDE8F88F04202F
:10983000FBE70920F9E700006C2B002010B50E4C67
:1098400003E0401C00E00020207020786178814215
:1098500010D022786188E068A36802FB010003EB66
:10986000C20153F83220898890472078A188884225
:10987000E9DAE6E710BD00006C2B002030B5CB0024
:1098800008339DB293074FF0000401D0072030BD8C
:10989000044B9A602A44DA605C701C70588099808E
:1098A000002030BD6C2B002030B5EFF3108172B674
:1098B0000D4A9468012324B10370002900D162B6D7
:1098C00030BD93604FF0E023D3F88051074C254022
:1098D0001560C3F88041D3F8844154605A17C3F827
:1098E000842100220270E8E7D04E0020FC06FFBD74
:1098F0000B498A68002A11D000280FD1EFF310809D
:1099000072B60B684FF0E022C2F800314B68C2F823
:10991000043100228A60002800D162B6704700003E
:10992000D04E002070B510480146456AC06A8C6C64
:10993000AC2801D024B106E0486B04442D1A02E0A3
:1099400001F00AFA04462A4621460848FEF789FD36
:10995000002807D001F066F829462046BDE870408F
:1099600001F01EBB70BD00005C47002000800700B6
:1099700030B504462C4995B04FF6FF704880012061
:109980008DF812004FF65960ADF81000224604A978
:109990000120A8DF002844D1244B0FCB8DE80F0015
:1099A000A11C684662DF00283BD120491C22603997
:1099B0000BA8FEF732FD1E4D142205F1C401A86864
:1099C0001290A0788DF84A002868139006A8FEF738
:1099D00024FD12A8069013A807902088231D06AA2C
:1099E0000BA9AADF00281CD11C2205F1D8010BA865
:1099F000FEF713FDE8681290A0788DF84A006868B9
:109A00001390142205F1F40106A8FEF706FD12A832
:109A1000069013A80790208804F10C0306AA0BA94E
:109A2000AADF15B030BD00002C2B002088D707001E
:109A300080D60700F0B585B0044614216846FEF7CD
:109A400005FD2078032308280BD12748C188491E2B
:109A500089B2C1808288002A3ED000293CD1C280D0
:109A600023702178607860228DF800208DF8011035
:109A70008DF802006078032101280AD00B2828D134
:109A800000F0C6FC8DF80300002000F0C9FC0421A2
:109A90001FE0207809281CD2DFE800F01B1B1B20E8
:109AA0001B1B051B2000D4E902706D46E91C66688B
:109AB00003F006FC044629193046C91C03F000FCDB
:109AC000044429193846C91C03F0FAFB2044C01C81
:109AD000C1B2684603F04AF805B0F0BDD4E90112FE
:109AE000684603F032F8F2E72C2B00202DE9F04114
:109AF0001349034600208A68D4071ED0114CA342A4
:109B00001BD04888A0F57F43FF3B10D042F00402F1
:109B10008A60132176DF00280FD10B4EC8254FF441
:109B20007A47741C3846A0476D1EFAD101E00878C8
:109B300074DFBDE8F04101F0EFBFBDE8F081000047
:109B40002C2B0020CCDA070090D6070038B5214C2A
:109B50000021227AD20701D0084638BDE0601E48B5
:109B600000F018FE0020009001F026FA88B91B488A
:109B700013DF70B901F0FAFF58B9684601F03AFFF7
:109B800038B96946012001F03FFF10B9684601F07D
:109B900089FF0028E1D101F0FBFA30B1104801F053
:109BA000EBFAA06840F00200A06000F04FFC002833
:109BB000D3D10B481C30FFF7DBFE0028CDD1FFF7D7
:109BC000ABFD0028C9D1A06840F00100A0600020D2
:109BD00038BD00002C2B0020D4DA070000800700DD
:109BE000E42F002070B50446011D008800226F4D4F
:109BF00086B021287ED025DC13287CD018DC0128F3
:109C00007AD010285BD011284AD14FF6FF706880B7
:109C1000287A400704D4FFF77FFD08B1FFF7BCFDA9
:109C2000E96800293CD006B00220BDE87040084732
:109C3000142878D01A2877D01F2831D16888091DB8
:109C400075DF62E0512870D02CDC222828D0232830
:109C500062D0242824D0502822D1554D34F8060F44
:109C6000A98888421CD1534800F05AFD060017D03D
:109C7000628904F10C01FEF7D0FB18224E496846B8
:109C8000FEF7CBFB049601956089ADF81400684699
:109C900001F0C6F9002803D03146464800F062FDC5
:109CA00006B070BD52287BD0552813D05628F7D166
:109CB000A0790028F4D11321688876DF25E0088890
:109CC0006880E96809B1012088473B4968887A398A
:109CD00075DFE5E7E188F72914D28807B0F1404F36
:109CE00011D0C91F89B2481EC21700EB927222F030
:109CF000030202E033E01CE036E0801A081A801DFF
:109D000081B200E0F7216888B5DF0028C8D006B02E
:109D1000BDE87040FFF740BD00920192A08800228C
:109D2000694690DF18E034E03AE021E0FFF734FDC7
:109D3000B6E721486A46903842F60521806A0090CD
:109D400002A801906888ADDF08B1FFF725FD002368
:109D50001A46852168887FDF0028E7D1A0E70092B6
:109D6000088869468FDFF7E70021688866DFCCE75F
:109D7000A079002894D021460D4802F005F900286A
:109D80008ED006B004F10801BDE87040084801F02B
:109D9000EDBF0024088822462346214686DFB4E72B
:109DA000002308881A461946B1DFAEE72C2B0020A5
:109DB00000300020D4DA070010D70700007800F048
:109DC0000100704713B90378012B01D001F003BBE8
:109DD000012070470022C32100F5187000F0B8B8C8
:109DE0002DE9F043A1B00446DDE9289520200F4677
:109DF000209098461646782102A8FEF727FB4121BD
:109E00002046FEF723FBB7F8940006EB061107EB9C
:109E10008101B04201D991F8965025701DB3012DF2
:109E200004D0022D0AD0032D13D116E0002249469A
:109E3000404600F08DF8C4F8010014E020A9601C31
:109E4000CDE900014B4642460A4902A800F098FEBF
:109E500048B1002021B0BDE8F083B1F89820601C23
:109E60009A31FEF7DAFA4A464146204601F0B3FA43
:109E7000F0E70000A8D4070010B500284FF000005C
:109E800006D004490870BDE81040034801F0ACB9A1
:109E900000F016FAE82A0020C1A207002DE9FC41D3
:109EA0000646C0074FF000050ED0104F00240122D7
:109EB000385D009500231146019501F0FAFC641C01
:109EC000042CF4D300F024F8B0070DD5074E00247D
:109ED000361D0022305D032300951146019501F0E7
:109EE000E8FC641C042CF4D3BDE8FC8198D4070082
:109EF0000249085C012101F011BD000098D407005F
:109F00000249085C002101F009BD000098D4070057
:109F100010B500242046FFF7EBFF641C042CF9D396
:109F200010BD10B543689C18446021B905E013F8D2
:109F3000010B01F8010B521EF9D2012010BD0000E7
:109F40000249CA6B4260096C816070475C4700201F
:109F5000F0B54FF0FF3622B11268D24300230A4D0C
:109F60000DE03246FAE7C45C62400824D70700D00F
:109F700037462F4087EA5202641EF7D15B1C8B42A2
:109F8000F1D3D043F0BD00002083B8ED10B50446F6
:109F90000068401C07D0204602F0BEFE21688142C6
:109FA00001D1012010BD002010BD000010B50B4CE8
:109FB00090B0607800280ED100F046FE20220849BB
:109FC000684600F061FE40236A460649064800F0F4
:109FD00097FD0120607010B010BD00005C2B0020C8
:109FE00058D40700084E0020C0D40700F0B514690B
:109FF00006468DB020681546271DE0B1022920D005
:10A000000A2000906B4609AA304602F06DFD002838
:10A010000FD009A901A8009A02F05CFB01AE96E8F6
:10A020000F0005AE86E80F00236869683A4605A868
:10A0300098470DB0F0BD0DB03046BDE8F04002F0DD
:10A04000BDBB6946304602F04FFB0028F1D02368C3
:10A0500069683A46684698470028EAD0029800287E
:10A06000F5D1019870600120E3E753689B7813F005
:10A07000C00303D0402B03D00020704700F002B88B
:10A08000FFF7B4BF2DE9FF410B4651680646144661
:10A090008878334D00F00F0210F0300055F8225050
:10A0A00006D0102806D0202808D0302856D13EE00F
:10A0B00022694DE061690120087047E0022B28D138
:10A0C000042A26D84FF0010869463046676902F035
:10A0D0000BFB00281AD009E00B89226903FB002240
:10A0E0006846A84770B13888401C3880029820B173
:10A0F000616838884A899042EED30198706002986E
:10A1000060BB02E04FF00008F7E7404604B0BDE84E
:10A11000F081D4E904300F890288498907FB0233B2
:10A120008A421BD2521C02801A46616810E00888DD
:10A130006169072A088009D1606801892069FEF7F2
:10A1400085F960682169C06802F0E9FA22696168EE
:10A1500004B03046AC46BDE8F04160470020D5E78A
:10A16000D8D9070038B5224801240168C90301D5B0
:10A17000811308E01F48016801F0F901A92904D101
:10A18000016801F05601016000241B4D286A012876
:10A190002CD14FF4405019494068884208D12346D9
:10A1A0004FF4805105F518706A6BFFF70BFEE8B1AC
:10A1B00000F0BEFD014623461148AA69FFF702FEE2
:10A1C000A0B119200090684601F09AFBD0F8100564
:10A1D0000099C84010F0010F08D00648001F006821
:10A1E00000F0F900B12801D0002038BD012038BDB1
:10A1F00000040040200500405C470020DBE5B15131
:10A20000FD4900204169002901D0C0680847704716
:10A2100010B508281BD2DFE800F004121A1A1A043D
:10A220001A040120FFF73AFE0020FFF769FE012023
:10A23000FFF766FEBDE810400220FFF759BE01207F
:10A24000FFF756FEBDE810400220FFF759BE10BDD3
:10A2500010B50446801E062810D2DFE800F00D037A
:10A26000030F09090A494FF4701000F0EDFA05E0F8
:10A270000120FFF701FE01E000F0DEFF0548416824
:10A28000002903D02046BDE81040084710BD00005B
:10A2900045A50700E82A002010B50446062801D08D
:10A2A000072C02D1002001F05FF804480168002962
:10A2B00003D02046BDE81040084710BD282B0020E1
:10A2C000BFF34F8F05480168054A01F4E06111436F
:10A2D0000160BFF34F8F00BFFDE700000CED00E011
:10A2E0000400FA052DE9FC4180461F4615460E463E
:10A2F00000240D4800F006FA38B11120BDE8FC81B9
:10A3000006EB043001F01EFB641CAC42F8D1064899
:10A3100000F0F5F9CDE9005733460022022140460E
:10A3200000F02AF80020E9E77C2B00202DE9F84313
:10A33000104D0F4680461E4691466946286800F03B
:10A34000B2F9040014D01C21FEF780F8012020711E
:10A35000C4F81490380BC4F80080C4E90260694660
:10A36000286800F0C1F902F09FFB0020BDE8F883E7
:10A370000420FBE704D807002DE9F04387B004462A
:10A38000DDE90E8980681D4616460F4600280BD071
:10A3900018216846FEF75AF802A88DF8007080E888
:10A3A0006003A1686846884707B0BDE8F08330B510
:10A3B0000446006887B00D46806800281FD0182129
:10A3C0006846FEF743F80195A0680590207910B122
:10A3D000012810D107E001208DF8000020690290CB
:10A3E000E068039005E002208DF80000E0680003BB
:10A3F000029060690490206881686846884707B0C9
:10A4000030BD0B2803D30B38C0B200F009B8704739
:10A410000249002208780A7070470000442B00208F
:10A42000014908700B207047442B0020014901208E
:10A4300008707047E82A0020014901200870704721
:10A44000242B00200123723000F0EEBF0EB59DF8E2
:10A45000080020F00F00401C20F0F00010308DF8B4
:10A46000080068466DDF002819D19DF80100401CE6
:10A470008DF8010068466CDF002810D10848007A8A
:10A48000800703D50748011D806901E006A1072068
:10A4900082B202A87CDF002801D105487ADF0EBD18
:10A4A0002C2B0020E42F0020446675546172670055
:10A4B00096D607002DE9F04781461D461646884688
:10A4C000494502D10020BDE8F087A8EB0900040B44
:10A4D00006F6FF704FF0000A070B00F0B7FAA5422E
:10A4E0002AD22C4628E0A74202D8BA46354601E0D7
:10A4F000A246250300225146484600F017FD0028D9
:10A50000E1D1681E00F003002A1A002341464846A4
:10A51000D21C00F021FD0028D5D10948A7EB0A077D
:10A52000761B016BA94429440163A844002000F074
:10A5300007FF5FEA000AC6D1002ED4D15046C2E719
:10A540005C4700200120FFF797BC000001494160F3
:10A5500000207047D8D7070010B50B4941600B4861
:10A5600000F0D0F868B901F04DFB08491C234FF406
:10A57000EE7208740448A1F5EE71001F006800F047
:10A580007FF8002010BD000008D80700C850002048
:10A5900002480068002800D0012070477C2B002072
:10A5A0000248007A002800D001207047C8500020DF
:10A5B00010B54FF44051144B4C6800F500509C42CC
:10A5C00004D042689A4201D1012200E000229C425C
:10A5D00018D144689C4215D10A78142A01D94969D6
:10A5E00000E00021094A0378B1FBF2F1142B01D9F4
:10A5F000406900E00020B0FBF2F0814201D001226E
:10A6000000E00022104610BDDBE5B15140420F00D2
:10A6100070B5054608680C464A6886682846314683
:10A6200001F09EFF6068286104F10C006861B07859
:10A630000221B1EB901F01D1241D2C6170BD0000DF
:10A6400000F0D8F94FF48051002000F011F940B922
:10A650000548C0F5FC2100F00BF910B9034800F0E3
:10A6600061F901F079FC00000080070011A20700E9
:10A6700010B5FDF71CFE08B1002010BD112010BD63
:10A6800010B531B1B2FBF3F403FB14241CB1092063
:10A6900010BD0E2010BD01600021416081608281EB
:10A6A000C381084610BD70B50C460546FDF7B4FDE4
:10A6B000002802D021882868084470BD10B50A8897
:10A6C00049888A4203D1FDF7E9FD012010BD002031
:10A6D00010BD70B50C460546FDF7C3FD002802D03D
:10A6E00061882868084470BD10B50A8849888A4284
:10A6F00003D1FDF7ADFD012010BD002010BD0021EC
:10A7000000F003B8012100F006B808B56A46FDF76D
:10A7100000FE009808BD08B56A46FDF7EDFD08BDCE
:10A7200038B5044600258DF800506846FFF7BCF8A0
:10A7300021686268086890420ED9401E086001785E
:10A74000238AE26801FB0325227A2168101AC0B22D
:10A750000A79824200D208719DF80000FFF7C8F81C
:10A76000284638BD38B5054600208DF800000C4657
:10A770006846FFF799F8E868298A201AB0FBF1F1DA
:10A780002A681068431C136001709DF80000FFF7F1
:10A79000AFF838BD10B530B1017A42680368891A44
:10A7A000C9B21A6006E00E2010BD03681A68541C76
:10A7B0001C601170491EC9B2F7D2006800210171F6
:10A7C000084610BD10B54FF0E0224FF0FF314FF4B6
:10A7D0008054C2F88011C2F8801200F0F9FB2046C4
:10A7E000BDE81040AFF3008010B504461448C0F532
:10A7F000FE2100F03DF808B1FEF7CEFF00F098FA18
:10A80000014610488069421EC2F30B02801A0144BF
:10A81000002001F6FF7100F02BF808B1FEF7BCFF35
:10A82000D4E90001002282F3148882F3108882F3B5
:10A83000118882F3138880F30888BDE81040084728
:10A84000008007005C47002070B5084D04460E46A6
:10A85000686802F02BFD002C06D03246214668685D
:10A86000BDE8704002F014BD70BD0000F42A002065
:10A8700030B50A0502D1B0F5FE2F01D9072030BD51
:10A88000094C2268082A01D3042030BD074B03EB92
:10A890000213C3F80008C3F804180220C3F808081C
:10A8A000521C0020226030BDF02A002000E0014050
:10A8B00070B5194D0024E86A2435012807D0A52871
:10A8C00008D0AA2809D0AC280AD0002070BDFEF715
:10A8D0003DFF0BE002F068F907E0FFF723F805E021
:10A8E00002F062F908B9FFF71DF80124284600F0CC
:10A8F00043FA0A4900200870094800F021FD08B118
:10A90000032070BD0120002CFBD00349096A0129F6
:10A91000F7D1022070BD00005C470020242B0020EE
:10A9200039A40700F8B52C4D6860192000906846DE
:10A9300000F0E6FF009A294900EB82000026C0F8EB
:10A940000017304600F056FC18BBFFF7B1FF20B1EE
:10A9500001281BD0022836D105E04FF47014FFF710
:10A9600001FC10B92CE04FF4A02400F06FF81C4A51
:10A9700020211820FEF782FF08B1FEF70DFF1948CD
:10A98000016801F0F901B12904D007E00120FFF7C7
:10A9900073FA18E0016801F04E01016000F0FEFA60
:10A9A00088B911492046FFF74FFF104800F0E0FA40
:10A9B00048B900BF00F036F8FEF740FF41DFF9E785
:10A9C00000F0C0FB08B10320F8BD2E70084800F06D
:10A9D0000BFCFFF7F7FEF6E7E82A00200C00030067
:10A9E000A42B00201C05004045A5070051A207002C
:10A9F0002DA4070010B540F6F8700168491C02D17B
:10AA0000074900F0B7FF40F6FC700168491C05D10A
:10AA1000BDE810404FF4FC2100F0ACBF10BD0000B9
:10AA20000080070010B501F08DF9002803D0BDE8C3
:10AA3000104002F0A3BC10BD034A93680A460146C9
:10AA40009860184602F024BCF42A002070B50E4D20
:10AA50002878002817D101F075F9012690B10B482C
:10AA60000468A4F54864962C00DA962402F086FC6B
:10AA700007492046FFF7E0FF4FF0E0214FF4803018
:10AA8000C1F800012E7070BD252B00200405014087
:10AA9000B9D3070040688068004710B542680830A5
:10AAA000527900F0F1F8002010BD2DE9F04399B083
:10AAB0001C4690460D460846DDF88090FFF7EAFFF9
:10AAC0006E6807467079A04200D804462246414687
:10AAD00011A800F015F97279494601A800F0D4F8E0
:10AAE00001AB224611A905F108000097FDF756FEBB
:10AAF00018B1002019B0BDE8F08348F24250F9E7E0
:10AB000070B516460C46054600F0E2F800280ED156
:10AB1000AA791946304600F0E8F8002807D13146F6
:10AB20002046FFF7BAFF002801D10149216070BD1E
:10AB30007052464D2DE9F8430C46DDE90857814631
:10AB4000984616460D49204600F0B6F8002810D168
:10AB50006068394640794200284600F0C6F800286F
:10AB600007D146B143463246214648460095FFF795
:10AB70009CFFBDE8F88348F21050FAE77052464D4A
:10AB80002DE9F0411D46DDE906871646044600F032
:10AB90002DF800280DD12A463146204600F03CF819
:10ABA000002806D13A4641462046BDE8F04100F073
:10ABB00002B8BDE8F08170B515460E46044602F0B5
:10ABC000CDFB002807D13EB160682968C268914278
:10ABD00005D248F2145070BD48F2135070BD83681E
:10ABE0002A4631462046BDE87040184710B550B19E
:10ABF00061B14160096804468847002802D10548D0
:10AC00002060002010BD48F2015010BD48F21050E5
:10AC100010BD00006E52464870B515460E460446FB
:10AC200002F09CFB00280BD146B155B160682A4662
:10AC3000314643682046BDE87040184748F210503E
:10AC400070BD002070BD00002DE9F0410B480C4D97
:10AC50000C4F401BC60801203870002406E000BFDE
:10AC600055F834008047002805D1641CB442F7D35E
:10AC7000022038700020BDE8F081000000000000D4
:10AC800000000000262B002070B514460D46064635
:10AC900000F036F8291930192246BDE8704000F05E
:10ACA0002FB830B50C46054600F035F82819214676
:10ACB000BDE8304000F02FB828B10068884205D0C8
:10ACC00048F24050704748F21050704700207047DB
:10ACD00028B139B10022C1E900201046704748F27E
:10ACE0001050704748F21350704720B1914205D080
:10ACF00048F21150704748F21050704700207047DA
:10AD00000244521E04E000BF11F8013B02F8013971
:10AD10008242F9D270470144491E05E002780B785F
:10AD200000F8013B01F801298142F7D27047000089
:10AD30004FF44050074A4168914207D18068411E54
:10AD4000C1F30B01401A00F6FF7070474FF48050BA
:10AD500070470000DBE5B15100B5FFF7E9FF054999
:10AD600089690A18401E0844C0F30B00101A00F647
:10AD7000FF7000BD5C4700200021016041608160E0
:10AD800001480163704700005C4700202DE9F04155
:10AD90009846214F16460C460546002301215BB11B
:10ADA000012B11D0022B1ED00020381AA0F5005024
:10ADB000A8421BD201221AE0FFF7CEFF8EB117493D
:10ADC000096A0129F1D00CE0FFF7B2FFB8F1000FDA
:10ADD00005D14FF44051124A4968914201D00121F6
:10ADE000E3E70021E1E74FF48050DEE7002242EA8A
:10ADF0000400884305D0022B03D25B1CDBB2022B7C
:10AE0000CCD912B10420BDE8F0811BB10348183041
:10AE1000FFF7B2FF0020F6E7008007005C47002044
:10AE2000DBE5B15170B504460078092811D2DFE89E
:10AE300000F0100510112510381013000D461D49A3
:10AE40000320C9688847606900F056FBFFF7D9FA0C
:10AE5000687070BD084628E00D46A18A206900F0A0
:10AE600027FBFFF7CEFA68702846FFF769F8E1681C
:10AE70000029EED02069BDE8704008470C460D4916
:10AE80000831081F00F052FBFFF7BBFA6070012881
:10AE9000DFD1002000F054FA0028DAD00A206070D8
:10AEA00070BD08464FF40071C160BDE87040FFF707
:10AEB00047B80000482B002070B51A4A05780124D5
:10AEC000936C092D2CD2DFE805F02B052B0B0F2BF3
:10AED000252B080000F084FF22E000F0F7FF1FE0C0
:10AEE0008B60106D48601BE0D2E91454566C2C1B2B
:10AEF000A64203D008204870012411E000245565C3
:10AF000054642146D36400F0A5FF07490420C968B2
:10AF1000884705E08B60106D48604FF48050C86032
:10AF2000204670BD5C470020482B002013460A468F
:10AF30000146014800F0F0BB902B002008B1034906
:10AF400000E003490022034800F0FCBB14D80700CE
:10AF5000E4D70700902B002008B5009313460A465B
:10AF60000146024800F086FC08BD0000902B00203E
:10AF7000084910B508600020FFF78EF9064800F078
:10AF80000DFA002804D1BDE81040034800F026B8AF
:10AF900010BD0000282B002099A207000020704758
:10AFA0001FB58908002201AB009283E807006846BC
:10AFB00018DF04B010BD00001FB5044B0FCB8DE8A7
:10AFC0000F00684618DF04B010BD000098D70700D6
:10AFD0004FF48050410408600020704710B5040011
:10AFE00011D00120FFF7AAFF00280BD100F04EFA84
:10AFF00000F0DEFA48B10949081F00F097FA01286D
:10B0000003D0032010BD072010BD04480838C460D9
:10B010000020FFF705FA002010BD0000502B002093
:10B02000816819B1024A1821FEF7B8BB07207047A2
:10B0300035B00700AFF3008030B587B00446182262
:10B040001F496846FDF7E9F920788DF8000022785D
:10B050001C4D0D2A25D2DFE802F0240B270B0B2410
:10B060000B240B2424240700E968072088471BE0F1
:10B0700020466946062A01D0012A01D1027C2A70A5
:10B080002A78012A05D0022A06D00020287005203F
:10B0900008E0FFF7C7FE07E0FFF70EFF20B907B093
:10B0A00030BD02208DF80100D4E9011268469047B6
:10B0B0009DF801000128F2D0E96805208847EEE7F5
:10B0C000C0D70700482B002038B105490160054969
:10B0D000416001210172002070470E20704700007E
:10B0E000E9B0070021B1070010B50C0001464FF090
:10B0F000110007D02278052A05D2DFE802F00F05FB
:10B100000D0F0F000E2010BD084600F051F800286A
:10B11000F9D10221217010BD112010BD082010BDF1
:10B120000246082041B10B78022B04D1022A05D037
:10B13000032A00D1112070470E20704700200322FF
:10B140000A70704770B50B480024D0F82413491CCE
:10B1500003D1D0F86403401C09D04FF4FE252846E3
:10B1600000F0F0FBC9220349284600F01BFC2046F2
:10B1700070BD00005C47002010B528B11C220349B7
:10B18000FDF74BF9002010BD0E2010BD64F3070041
:10B1900010B5064C00221821201DFEF7D9FE2168AB
:10B1A000814201D1012010BD002010BD64F30700D1
:10B1B00070B50C4D0400D5F8640305F5597503D03E
:10B1C000401C03D0082070BD0E2070BD0022182145
:10B1D000201DFEF7BDFE206007222146284629DFFC
:10B1E00070BD000000F00700014901F08BBD0000B8
:10B1F00000F0070010B5FFF7A1FE30B900F01CF811
:10B20000002000F09DF8002800D0032010BD0000B1
:10B2100010B5FF224FF400710648FDF710F90548FC
:10B2200020212438FDF712F9024900205C39086317
:10B2300010BD0000B84700202DE9F0472E48FEF76A
:10B24000A5FE2E4E074634682046FEF79FFE4FF0BF
:10B25000010A4FF0000958B16068012806D0204665
:10B26000FEF7B8FDD4F85C12884201D1012500E058
:10B270000025234C4FF002084FF460719FB10A463D
:10B280001D492046FDF7C9F89DB136682546542270
:10B29000311D281DFDF7C1F84FF4327206F15C0133
:10B2A00005F15C0003E015B30A4615483168FDF767
:10B2B000B4F86068012818D11249402201F5E47001
:10B2C000FDF7ABF80F491C22403101F5E470FDF7A2
:10B2D000A4F884F8609284F8A1A20B4884F8E29262
:10B2E000E169C0F82210C4F80480BDE8F087044882
:10B2F000FDF7ACF8F7E7000000F00700582B00203E
:10B300005C470020B8480020DC49002070B50546A5
:10B31000094801F001FD084C20602046FEF75AFD67
:10B32000C4F85C02A4F5E0632A462146BDE87040FB
:10B33000024801F0F6BC00005C47002000F0070066
:10B3400070B505460020FFF7E1FF040003D1034973
:10B35000284601F0D7FC204670BD00005C47002065
:10B360004FF48050704700002DE9F041074609482E
:10B37000094D401BC6080020044607E005EBC40049
:10B38000416838468847002802D1641CB442F5D38E
:10B39000BDE8F081D4DA0700CCDA07002DE9F041EE
:10B3A00007460948094D401BC6080020044606E030
:10B3B00055F8341038468847002802D1641CB4423E
:10B3C000F6D3BDE8F0810000D4DA0700CCDA07003C
:10B3D000012201F021BA38B5144602780B467AB141
:10B3E000012A04D0022A0DD0032A1BD112E0D0F882
:10B3F0000150002221461846FEF7AAFDA84211D1AD
:10B40000012038BD01B02246BDE830400023401C79
:10B4100000F00AB8411C40220020009400F0F2F82D
:10B420000128EED0002038BD2DE9F041AAB0054634
:10B430002020884628901E4617460124782102A81D
:10B44000FDF704F8FEF7B2FD2EB12022294620A810
:10B45000FFF756FC20AD28A90A48CDE900013B467C
:10B460004246094902A8FFF78BFB28B9202229464A
:10B470000448FCF7F6FF00B100242AB02046BDE8DE
:10B48000F0810000B04E0020A8D4070010B5064897
:10B49000064C806B20B101F02DFE08B1012000E0C8
:10B4A0000020207010BD00005C4700205C2B0020B5
:10B4B0002DE9F0410F4C07460D46E06BA26B0126CB
:10B4C0004119914201D9032610E00A492A465C310C
:10B4D00008443946FCF7A1FFE06B064A2844E063C4
:10B4E000403229463846FEF733FD20643046BDE839
:10B4F000F08100005C47002070B504004FF00105AA
:10B5000004D0B4F5007F03D9042508E0032506E044
:10B51000044900200870FFF77BFE03488463284637
:10B5200070BD00005C2B00205C4700202DE9F0413D
:10B5300006461D480F46C16B806B814201D008242E
:10B540002FE01A4D287840B1FFF706FC30603946ED
:10B55000E86801F0D7FE044623E001F0CBFDF8B126
:10B5600000F02CF80446002030603860012C0FD128
:10B570003946E86801F0C6FE0446012808D138685B
:10B58000012700213B460A46FFF700FC18B10424BE
:10B59000FFF73EFE05E0FFF7DFFB30602F7000E0B5
:10B5A00005242046BDE8F0815C4700205C2B00208C
:10B5B00001480078704700005C2B002038B50F4C24
:10B5C000251D002094F86C31014602463BB194F8E9
:10B5D000D802B4F8DA2204F5B87504F53771084BCF
:10B5E0009C6800945B6800F00DF8012804D1281DC8
:10B5F000BDE8384000F050B838BD0000DC4A0020FB
:10B600005C2B00202DE9F041A2B0064620200D461B
:10B6100020901F461446DDF8A080782102A8FCF790
:10B6200015FF00202190FEF7C1FC25B12EB1162098
:10B6300022B0BDE8F0811320FAE720A91448CDE933
:10B64000000143463A46134902A8FFF799FA08B9A0
:10B65000402C01D00A20EBE70D482246294640380D
:10B66000FCF7DBFE0A4820214038FFF71AFB0848A8
:10B6700040214038CDE90001A0F14801044A21A849
:10B68000209BFFF757FA08B10520D1E70120CFE74B
:10B69000904E0020A8D4070070B5044690F85400DE
:10B6A000012570B394F8550028B1012803D0022871
:10B6B00001D003282AD194F86E00032801D0142564
:10B6C00025E0207AE8B1E068342801D011251EE099
:10B6D000204601F0B5FA68B1207898B194F8551079
:10B6E0000C4849B1012907D06168C06881420ED871
:10B6F00010250CE012250AE061688068814206D2BC
:10B70000F6E703E094F85500012800D00F252846FD
:10B7100070BD00005C4700202DE9F0410446406800
:10B7200015461E4602680F466A432046FDF7B2FFE3
:10B73000206833462A46D0F810C039462046BDE876
:10B74000F041604701600B68114618472DE9F04150
:10B7500028B1016819B1C969BDE8F04108470D4D2C
:10B760000D480024461B14270DE000BF04EB8400A5
:10B7700005EB8000016829B1C969884710B1012033
:10B78000BDE8F081641CB6FBF7F0A042EED80020C3
:10B79000F6E70000902B0020A42B00200448012194
:10B7A0004174007A08B10020704701207047000002
:10B7B000C8500020012801D0032808D104490022E4
:10B7C00001284A7400D00020087401F01FB97047A6
:10B7D000C850002070B50146022801D0032943D18A
:10B7E000224C207A00283FD0012831D002282FD1C6
:10B7F0001F4800230229006802D0032928D119E03C
:10B80000E360027912B1012A22D10BE0D0E905658B
:10B81000721B142A00D314222A4482614569AA4269
:10B820000ED015E00169491C0161426991420FD1B6
:10B83000237213E0E268521CE260082A08D9E36030
:10B84000237202290AD00D21FEF7B1FD01F0D4F8D0
:10B85000607C28B1BDE8704000F0DAB90021F3E760
:10B86000BDE8704001F0D2B870BD0000C8500020A3
:10B87000802B00202DE9F84304461D4616460F464E
:10B880000846DDF82080FDF7FFFE3046FDF7FCFEA0
:10B890002A4639462046FDF7FDFECDF80080206897
:10B8A0002B463246D0F80CC039462046E047BDE86A
:10B8B000F8832DE9FF411C46DDE90A7815460E465E
:10B8C000684600F00FF846EA450141EA840141EA82
:10B8D000072242EA0841009A00EB8200C0F80017F4
:10B8E000BDE8FF810168202902D24FF0A0407047D7
:10B8F00001F01F0101600148704700000003005083
:10B900000168202902D24FF0A040704701F01F01CA
:10B9100001600148704700000003005038B5012461
:10B920000090684631B1FFF7DDFF00998C40C0F808
:10B93000084538BDFFF7D6FF00998C40C0F80C458C
:10B9400038BD0000094902220A60BFF36F8FBFF3C0
:10B950004F8F0A1D106006480268002AFCD00020A4
:10B960000860BFF36F8FBFF34F8F704704E501404E
:10B9700000E40140094A01231360BFF36F8FBFF356
:10B980004F8F0160064801680029FCD0002010603C
:10B99000BFF36F8FBFF34F8F7047000004E5014086
:10B9A00000E4014070B50E4C01232360BFF36F8F9C
:10B9B000BFF34F8F00230B4D08E000BF51F8236009
:10B9C00040F823602E68002EFCD05B1C9342F5D318
:10B9D00000202060BFF36F8FBFF34F8F70BD00005A
:10B9E00004E5014000E4014008B5002242504058FF
:10B9F000009008BD20B1034909680160002070472C
:10BA00000E207047ACD90700FEB506460D46084625
:10BA1000FFF7F0FF002844D100240094019401278F
:10BA200006208DF80060ADF8040002948DF80270D5
:10BA3000694620202A6869DF00948DF801708DF82E
:10BA40000240019402948DF80340694640202A6820
:10BA500069DF00948DF80060F720ADF802000194D2
:10BA60000294694623202A6869DF009401940294B5
:10BA70008DF80070694601202A6869DF4FF4B060D4
:10BA80000090019402946946A1202A6869DF00941D
:10BA9000019402948DF800406946A0202A6869DF6D
:10BAA0000020FEBD60DF002802D1024A0121117092
:10BAB000704700008B2B002030B51548ADF5017D97
:10BAC0000078002821D04FF4FA7500BFADF800527D
:10BAD00080A9684661DF38B1052816D00DF5017DD3
:10BAE000BDE83040FDF758BE6C460A497DA800F01D
:10BAF000BBF806E0D0E90021204690477DA800F081
:10BB0000CAF87F980028E1D0F4E70DF5017D30BD3B
:10BB10008B2B0020B0D90700F8B5134C2078C0B1AA
:10BB20000120A07001F0C0F8112814D0022001F00B
:10BB3000D3F800258DF800506846FDF7B5FE11DFFB
:10BB4000064625709DF80000FDF7D2FE2EB1304666
:10BB5000F8BD0820F8BD0020F8BDA57001F07EFA00
:10BB6000032001F0B9F8F6E7882B00207CB5194CCA
:10BB7000207808B108207CBD0120A070002001F0D1
:10BB800093F8112819D0002001F0A6F812480026D9
:10BB9000006801908DF800606846FDF785FE0F494A
:10BBA00001A810DF05000AD0002020709DF80000D9
:10BBB000FDF79EFE2DB128467CBD00207CBD0120F6
:10BBC000F3E7A670667001F069FA012001F084F8CD
:10BBD000F3E70000882B002044D907009597070061
:10BBE0000EB50749684600F03FF805E0D0E90010BF
:10BBF0008847684600F04FF802980028F6D10EBD3D
:10BC000060D907000148007870470000882B0020A9
:10BC10000548817819B1007818B1FFF77DBF082079
:10BC20007047FFF7A3BF0000882B00201FB56846B0
:10BC30004BDF30B1052814D004B0BDE81040FDF74B
:10BC4000ABBD084901A800F00FF806E0D0E90021DB
:10BC50000098904701A800F01EF803980028E6D04D
:10BC6000F4E71FBDCCD90700016009684160AFF35C
:10BC7000008010B5D0E900215368994201D100211C
:10BC800004E0D1E90034A34202D01946816010BD1E
:10BC900008314160F0E7816800290BD002689268A2
:10BCA0000A44826041684B689A4203D1083141607E
:10BCB000FFF7DFBF704700002DE9F041044613484D
:10BCC000134BC01A0C21B0FBF1F6A0694FF0FF3105
:10BCD00010F8022C02B92169002011E000EB4005A8
:10BCE00003EB85052F68974209D14F1C02D06F687E
:10BCF0008F4204D194E80F00AD68A84703E0401CD0
:10BD0000B042EBD301202060BDE8F08124DB0700C6
:10BD100018DB070010B5144612680830202A02D23A
:10BD200048F2145010BD002201F023F80028F9D188
:10BD300020202060002010BD083001F0A3B808309A
:10BD400001F062B902480068002800D00120704765
:10BD50000004014003490860034801680029FCD041
:10BD60007047000004E5014000E4014030B587B0B1
:10BD70000C460546182217496846FCF74EFB217B06
:10BD800015488DF800100195012906D0022917D019
:10BD9000062919D1607B049016E08188C180607B00
:10BDA0000490217CE08961F31F40617C40EA0160DE
:10BDB00005900498012807D10848FFF7D5FA03E059
:10BDC000B4F80D108180C1806846FFF729F907B0EB
:10BDD00030BD0000E8D607002C2B0020CCDA07008D
:10BDE0002DE9F0410C460546FFF7E2FB0826B8B105
:10BDF0006969032041B3154A154B0F0505D0576DEE
:10BE0000D3F808C00F4467451ED1B1F5805F01D952
:10BE1000042019E0506DD3F808C04718674502D9CF
:10BE20006670BDE8F0815164D16C10659164106357
:10BE300069695A6801F6FF711044090B0022FFF787
:10BE400075F80028EDD005206070EAE75C47002017
:10BE5000482B002010B5044686B00020FFF776FC82
:10BE600030B1154A18212046FDF798FC06B010BDE8
:10BE7000182212496846FCF7D0FA1148026D1148A1
:10BE800081688A4210D14068FFF7A2FA8DF801005C
:10BE9000FEF7B7FA8DF80100D4E901126846904721
:10BEA0000948FFF74DFAE1E701208DF80100D4E9D8
:10BEB000011268469047D9E755BE0700A8D707008A
:10BEC0005C470020482B00204DBF07002DE9F041C2
:10BED0000E460446FFF76CFB60B11A4DD5E914011C
:10BEE000401AA18A6A6C0844904205D903207070F8
:10BEF000BDE8F0810820FAE7134A286B52688718DA
:10BF0000104A20694832FEF723F8D4E9033180460D
:10BF1000A28A3846FFF720F820B1D4E90310BDE823
:10BF2000F0410847A18A286B08442863A18A286D3C
:10BF3000C5F8488008442865C6F80880286D7060F8
:10BF4000D6E700005C470020482B0020014906206E
:10BF5000C9680847482B0020BFF34F8F0548016888
:10BF6000054A01F4E06111430160BFF34F8F00BF48
:10BF7000FDE700000CED00E00400FA050146014871
:10BF8000FEF7F0BBD4DA070030B58A1D8B79083193
:10BF900087B0022B33D153888489A3422FD1127AE0
:10BFA000012A2CD1184C0DF1040C3CCC8CE83C003F
:10BFB0000A89ADF80C204A890C3104911249ADF878
:10BFC0000E208039114C096A0591CDF818D0018AEC
:10BFD00005AA6088ADDF18B96846FDF7EFFE38B1F5
:10BFE0000020ADF8080001A96088B0DF50B106E07C
:10BFF00040F2FD10ADF8080001A96088B0DF002014
:10C0000007B030BD0120FBE700D707002C2B002034
:10C01000F8B50D4614460646694600F05DFA00285C
:10C020000FD0009BB3F5803F0AD2981C834207D8FB
:10C03000A9780222B2EB911F02D02989814201D254
:10C040000020F8BD2380A11C3046009A00F07AFB46
:10C05000F8BD114600F0D5B8114600F0E7B8F8B5C4
:10C060000C4615460646694600F036FA00280CD004
:10C07000009A501C904207D3A1780223B3EB911F82
:10C0800002D02189814201D20020F8BD29463046E4
:10C0900000F058FB009A0021A954F8BD2DE9FF419A
:10C0A0000C46CE6817460546694600F01DFB002881
:10C0B0000ED0E06800280BD0A0783A46C0F30110FB
:10C0C00002283146684606D000F0DEF80199696022
:10C0D00004B0BDE8F08100F085F8F7E77CB50D46C7
:10C0E0001446694600F095F9002820D028890828D0
:10C0F00006D0042809D002280AD001280CD015E067
:10C10000DDE90001C4E900010AE00098206006E0D2
:10C11000009800B2208002E0009840B22070C11761
:10C12000DDE9002350405940084301D000207CBD88
:10C1300001207CBD7CB50D461446694600F0A7F988
:10C14000002820D02889082807D00021042809D0F9
:10C1500002280AD001280CD014E0DDE90001C4E96E
:10C16000000109E00098206006E0009880B220807D
:10C1700002E00098C0B22070DDE900235040594031
:10C18000084301D000207CBD01207CBD7CB50D465C
:10C190001446694600F07BF9002820D02889082839
:10C1A00008D00099CA1704280BD002280CD0012807
:10C1B0000DD013E0DDE90012C4E900120846134671
:10C1C00008E00846216004E008B2208001E048B29F
:10C1D0002070C31748405340184301D000207CBD55
:10C1E00001207CBD70B50D46064614461146284612
:10C1F00000F095FA224629463046BDE8704000F02E
:10C2000043B838B50C460422694600F09BFA002872
:10C210000BD09DF80210BDF8000061F31F409DF89F
:10C22000031040EA01602060012038BD1CB50C46B7
:10C230000822694600F086FA002824D09DF80110F3
:10C240009DF800209DF80230080E42EA012242EAE1
:10C25000034240EA13409DF803309DF8041040EA81
:10C26000132008439DF8051042EA036240EA0120CA
:10C270009DF8061040EA01409DF8071040EA016071
:10C28000C4E9002001201CBD2DE9F04F05469DB0FA
:10C2900000200F90064610904FF0FF3A01A800F0E2
:10C2A0005FF94FF0010B0DF13C0983E012AB6A46D8
:10C2B0000BA9284600F0CAF850B101A8009900F077
:10C2C00060F960B10298807810F0300F54D061E0CE
:10C2D0009DF84800002871D11DB0BDE8F08F00988E
:10C2E000B04243D3029C01AE0298807800F00F0068
:10C2F000082812D0304600F05BF90298A042F3D132
:10C3000056460098B04231D3D5F8088007909DF882
:10C310002C000E900598046821E002980688F0E74A
:10C32000206807682FB1214628460E9B079AB84718
:10C3300012E01195216807980E9F8968098881424B
:10C340000CD1214617A8FEF763F984F80CB017AAA0
:10C3500039461198FDF789FE0028BDD0A46814B1B4
:10C36000A9684145DCD0A968414523D19DF82C102E
:10C37000284600F023FA1BE0039840280AD200F078
:10C380001F000BFA00F20398400959F820301343BC
:10C3900049F82030EC682CB101AB9DF82C202846E0
:10C3A0000099A04701AA9DF82C102846FDF75DFED4
:10C3B000002891D0A86800287FF478AFDDE9020456
:10C3C000857801A800F0F4F80028F7D115F0300FB7
:10C3D00003D10298008800B1641CC4B10020494612
:10C3E00005E000BF51F82020521C0ED1401CB0EBDC
:10C3F000541FF7D3600959F8201004F01F00C0F152
:10C4000020022AFA02F0814201D0002064E70120D4
:10C4100062E71CB50C46694600F039F8002814D0D4
:10C42000DDE90002C10709D051084FEA30006FEA88
:10C4300000026FEA0100C4E9002004E051084FEA5D
:10C440003000C4E900014FF001001CBDF8B50746FB
:10C450000020187008700E4610601C46154669468C
:10C46000384600F039F801004FF0010009D000997A
:10C4700059B1C8082860009800F00700307001200A
:10C48000F8BDB96809B10020F8BD2070FBE72DE9BF
:10C49000F8430026884681463446354604E0402E5F
:10C4A00002D30020BDE8F8836946484600F076F9DB
:10C4B0000028F7D09DF80070324607F07F00C10FCA
:10C4C000FBF79CFF29430443F61D0D463806E6D4CE
:10C4D000C8E900410120E5E7F8B50E460746694680
:10C4E00000F05CF900280AD09DF80040200616D51F
:10C4F000072504F07F0403E0202D01D30020F8BDC0
:10C500006946384600F04AF90028F8D09DF8001036
:10C5100001F07F00A8400443ED1D0806ECD4012083
:10C520003460F8BD10B559680B4AC968914212D100
:10C530000A4AD0E90110D2E90134234301D0002096
:10C5400008E011F8013BA0F101001B06F9D4C2E993
:10C5500001100120907010BD30D507005C2B002029
:10C56000C26000230160C0E901138B881A44026194
:10C57000B1F906301A4442610888002800D0012031
:10C58000704770B545680E46044660680188B14240
:10C5900006D1807800F00F00082801D0012070BD7E
:10C5A000204600F005F86068A842EED1002070BD7A
:10C5B00030B541680A885AB101F1100343600A8A14
:10C5C00042B18C780A89C4F30115032D07D00BE022
:10C5D000002030BDC2680168FFF7C2FFF8E79D7810
:10C5E000C5F30115032D06D00225B5EB141F08D1A4
:10C5F0004C89624309E08D8804690022641B046150
:10C6000003E0B5EB941F00D10422897811F0300FBC
:10C6100002D18168491C81609C88016921441144D0
:10C620000161B3F9062011444161012030BD30B5EC
:10C630004168002487B0897801F00F02082A11D0E0
:10C640008A091ED00222B2EB911F09D10269C1F3FF
:10C6500001110229146001D0032901D1406904802D
:10C6600007B030BD0069056808E02C7329466846AC
:10C67000FDF7CEFF6846FFF7DAFFAD68002DF4D175
:10C68000EEE7C1F30111012912D00229E6D00329F6
:10C69000E4D04268917801F00F0107290BD0D168EE
:10C6A00081B11289006907B0BDE83040FBF7B5BE23
:10C6B00041690C70EDE70169D06807B0BDE8304012
:10C6C00000F02DB81189006907B0BDE83040FBF7D4
:10C6D000BDBE000010B5034B002408C080E8160062
:10C6E00010BD0000239F070038B50D46044669467B
:10C6F000FFF7F2FE00280BD0D4E90002D4E90213C0
:10C70000C5E90002C5E902130098814201D2002068
:10C7100038BDA860A168081AA060012038BD00B526
:10C720000A4687B001466846FFF71AFF002807D07F
:10C730006846FFF77CFF6846FFF73AFF0028F7D10D
:10C7400007B000BD7FB514460546A9B9124A28684E
:10C75000904208D110E0102269462846FFF7F2FF08
:10C76000002807D0103C102CF5D8224669462846F0
:10C77000FFF7E8FF04B070BDA868A04201D2002016
:10C78000F8E72B682246284698470028F2D0A86888
:10C79000001BA8600120EDE7239F070010B50446A9
:10C7A0008068002809D02368012220469847002885
:10C7B00003D0A068401EA060012010BD38B5002441
:10C7C00039B1012912D0022912D005291DD000202B
:10C7D00038BD0546012269462846FFF7B3FF90B1F0
:10C7E0009DF800000006F5D4012038BD08220DE0B8
:10C7F00005466946FFF770FE28B100212846009AD9
:10C80000FFF7A0FF38BD204638BD0422BDE8384000
:10C810000021FFF797BF00002DE9F04F81462C481B
:10C8200017460E46C5680A4693B001244946284675
:10C83000FDF708FEDFF89C80A24670B195F8550020
:10C8400068B100F00101C0F340024B462846CDE933
:10C85000006700F043F8D8B11BE0172419E0CDE9D8
:10C86000006A4B460022294602A8FDF7B9FA4FF0AC
:10C87000000B68B10FB3412202A91748FBF7CDFDA9
:10C88000C8F820B0C8F82CA06968C8F8081017E0EC
:10C8900005246FB1012C13D00E482430FEF76CFA3A
:10C8A000FEF7B6FCC8F8489013B02046BDE8F08FFC
:10C8B000012C02D0FEF7ACFCF6E7C8F814A0F3E7B1
:10C8C000002231464846FDF743FBC8E90960E7E727
:10C8D0005C2B00205C470020FD4900202DE9F0473B
:10C8E000A4B08946DDE92C5A0446984616464421F0
:10C8F00002A8FBF7ABFD442113A8FBF7A7FD4746B1
:10C90000B9F1000F38D008F50050384A4368A16DDE
:10C91000934255D14B1EC3F30B03C91A41F6FF7363
:10C92000D0F808C019448C454AD34FF440514B68A5
:10C9300093420DD10A78102A01D9096900E000213B
:10C940000278102A01D9006900E00020814237D125
:10C950004046FDF72DFE00B18EB30121A06DCDE95B
:10C96000000143460022214602A8FDF739FA0028BB
:10C9700027D0A06D07442D1A56B10020CDE90050F4
:10C980003B464A46214613A8FDF72AFA002818D04C
:10C99000BAF1000F28D0164DB9F1000F19D040465A
:10C9A000FDF706FE18B105F11800FEF7E5F9412282
:10C9B00002A91048FBF731FD36B1AC2005E0FFE7D6
:10C9C000002024B0BDE8F087A520E862A06D686370
:10C9D00001E0AA20E8623EB10648412213A9823054
:10C9E000FBF71BFD6068E8600120EAE7DBE5B15179
:10C9F0005C470020BC490020034802490068FDF75D
:10CA00005DBE0000842B002004D807002DE9F04112
:10CA1000224C0025224E207A012730B92148311DB1
:10CA20000068FDF756FE306038B102202072316890
:10CA3000087928B101281CD114E06560BDE8F081B7
:10CA4000D1E90503C01A142800D31420B7EB900FC6
:10CA500001D2820800E001220869C968184419441B
:10CA600029DF03E0D1E90301084428DF58B1112888
:10CA700012D003213068FDF79AFC25726560BDE88D
:10CA8000F041FFF7B9BF207C0028D7D1BDE8F041C5
:10CA900000210220FEF79EBE2772CFE7C85000207B
:10CAA000802B002004D8070010B5074C201DFDF78F
:10CAB00029FE002806D1607C002803D1BDE8104083
:10CAC000FFF7A4BF10BD0000C850002010B51046ED
:10CAD0001A46FBF7A2FC002010BD10B510461A46FE
:10CAE000FBF79BFC002010BD2DE9F0411E681C46A1
:10CAF0001546074621B1012918D0052923D119E08F
:10CB000000202060401C2060B0421CD80122294631
:10CB10003846FFF717FE002806D015F8010B00066F
:10CB200001D52068EEE70120BDE8F081082002462B
:10CB3000186002E004200246186029463846BDE825
:10CB4000F041FFF7FFBD0020EEE770B516460A463C
:10CB50000446C11C104600F0B3FB0546611930467F
:10CB6000C91C00F0ADFB284470BD000003B5094AA4
:10CB700085B0D2E91612CDE9001207498989ADF8CE
:10CB8000001006A9CDE90210044869464088AEDFCE
:10CB900007B000BD80D60700003000202C2B0020FD
:10CBA000084670470846704770B5FEF7D9FB114A32
:10CBB000114E136B546B916CE21A551EC5F30B05A5
:10CBC000521B42F2040518446D5802F6FF72B5423A
:10CBD00001D0032070BD1944A34201D1002070BDD3
:10CBE0000823FDF767FC0028F9D1BDE87040FEF787
:10CBF000A7BB00005C470020DBE5B151F0B505465E
:10CC0000002003464FF440540C4E4FF6FE7712E0DE
:10CC1000D4F804C0B44505D155F823C0B4F80CE0ED
:10CC2000F44504D02AB155F823C0BC4501D10120F8
:10CC3000F0BD5B1CDBB28B42EAD3F0BDDBE5B1514A
:10CC400010B54FF44051174B4A68018A9A4221D1DE
:10CC500071B100F11403426990F8550062B10428E3
:10CC600008D00022BDE81040C9B21846FFF7C6BF81
:10CC7000002010BD0122F5E710B1012808D1F7E727
:10CC8000012905D9C9B200221846FFF7B7FFEFE71F
:10CC9000012010BD11B141690029E9D100780028B7
:10CCA000F6D110BDDBE5B1513EB5044609496846F1
:10CCB000FEF7DAFF08E000BFD0E9002120469047E8
:10CCC00030B16846FEF7E7FF02980028F4D13EBD78
:10CCD00011203EBD48D907003EB5044608496846C4
:10CCE000FEF7C2FF07E000BFD0E9002120469047D1
:10CCF0006846FEF7D0FF02980028F5D13EBD00003F
:10CD000054D9070002460348014B006800F009B8F7
:10CD1000DC430020582B002000225821001DFDF785
:10CD200017B92DE9F04114464FF460751E460F46C1
:10CD300080462A46FBF795FB30B100220121404690
:10CD4000FEF7F4F898B905E00CB10020A0470020E8
:10CD5000BDE8F0812A4639463046FBF75EFB2346A4
:10CD60002A4631464046FEF7F7F80028F0D0032067
:10CD7000EEE770B516460D46040007D035B1206CBD
:10CD8000802200213828225403D307E00E2070BDF2
:10CD90002154401C3828FBD30BE02154401C402870
:10CDA000FBD32146084600F097F838212046FBF7D0
:10CDB0004DFB216CD4E912304A0FC90038345918A0
:10CDC0005041C4E90410227CE2710A0A42EA00627E
:10CDD000A2710A0C42EA00426271020242EA116048
:10CDE00020716069E070010AA170010C6170000E91
:10CDF00004F838092146084600F06EF84FF00002AA
:10CE0000EEB1E06ED100C840A854A36ECB40A81884
:10CE10000371636ECB400372236ECB400373E36DEB
:10CE2000CB400374A36DCB400375636DCB40037699
:10CE3000236DCB40521C0377042AE2D31FE0182352
:10CE40005042216D03EBC000C140A954666DC6403D
:10CE5000A9180E71A66DC6400E72E66DC6400E731F
:10CE6000266EC6400E74666EC6400E75A66EC6402F
:10CE70000E76E66EC640521C0E77042AE0D30020E0
:10CE800070BD0000A8B100210164C0E912110A4977
:10CE900001650A4941650A4981650A49C1650A492E
:10CEA00001660A4941660A4981660A49C16600204D
:10CEB00070470E207047000067E6096A85AE67BBC1
:10CEC00072F36E3C3AF54FA57F520E518C68059B6C
:10CED000ABD9831F19CDE05B2DE9F04FC8B000221C
:10CEE00013466F46CC181B1D2588A6786DBA2D04F5
:10CEF000E47845EA0625254347F82250521C102ABB
:10CF0000F0D31BE007EB820151F8083C4FEA734471
:10CF100084EAF34484EA932451F83C3C4FEAF31545
:10CF200085EAB34585EAD303234451F81C4C51F8F4
:10CF3000401C2144194447F82210521C402AE1D3D6
:10CF4000036D4793416D4691846D4594C26D449243
:10CF50009246026E4392456E4295A946856E419572
:10CF6000C66E4096B34600264FEAB21787EAF2270C
:10CF700087EA726C02EA090725EA020887EA0807CD
:10CF8000BC44204F57F8268008EB0B07BC445DF8E3
:10CF90002670AB460CEB070E4FEAB30787EA7337F0
:10CFA00087EAB35C81EA04074D4601EA040891462A
:10CFB0001F400AEB0E02A24687EA08070C46BC4453
:10CFC0001946761C0EEB0C03402ECDD3479E3344FE
:10CFD0000365469B194441654599214481654499FF
:10CFE0005144C165439911440166429949444166DF
:10CFF00041992944816640995944C16648B0BDE8C9
:10D00000F08F000034D807002DE9F04116460F4696
:10D01000040004D006B317B10025A8461AE00E207C
:10D02000BDE8F081216C785D6054206C401C206468
:10D0300040280ED121460846FFF74EFFD4E91201E1
:10D040004FF40072801841F10001C4F84080C4E937
:10D0500012016D1CB542E5D30020E1E710B51620A2
:10D06000FCF700FB48B10C4882684FF4800152B1D4
:10D07000016821F48001016010BDBDE8104042F25A
:10D080000100FCF789BB4FF0E020C0F88011BFF32E
:10D090004F8FBFF36F8F10BDD04E002010B51620FC
:10D0A000FCF7E0FAA0B1114890F800044009082804
:10D0B00011D20121814011F0EC0F0CD00C48826894
:10D0C0004FF480016AB1016841F48001016010BD34
:10D0D00042F2010001E042F20200BDE81040FCF71C
:10D0E0005BBB4FF0E020C0F8001110BD16E000E07F
:10D0F000D04E00207FB52A4800F15C01826B684663
:10D10000FFF7E8FA274E9DE8070006F11C03274CBD
:10D1100083E8070019462448C8600020A0706060BA
:10D12000A0604FF44771A6F54070FBF78FF9A6F5A4
:10D1300040721F4902F54770FFF754F800282BD0C2
:10D14000A07858B3A6F5407090F86C1100290178CA
:10D150001CD019BB90F8720100B3D4E90112A6F5F6
:10D16000C6756846FFF7B6FA9DE80F001C3686E8DC
:10D170000F004FF4B2712846FBF768F92A460D49B3
:10D180003046FFF72FF8002806D003E031B1807950
:10D1900020B1094D0120E56004B070BD0020FBE71F
:10D1A0005C470020DC4D002025C507005C2B0020DB
:10D1B00050D6070030D50700E44A002070B503467A
:10D1C0006FF07F40814200D20846124DD5F8042509
:10D1D0000244081A411E22F07F425860952902D26B
:10D1E0009630963A58601C7B05EB8400C0F84025C9
:10D1F00009494FF4F86088474FF4A07000EB8401B0
:10D200002846FEF7F1FB4FF48030A040C5F8040338
:10D2100070BD000000400240A1D4070070B5174E59
:10D220003078002829D1164800680125C0F3004055
:10D2300008B914480560144C4FF480712046FEF77D
:10D24000D3FB4FF4A0712046FEF7CEFB4FF4A27142
:10D250002046FEF7C9FB0D49A02081F800040B49C8
:10D2600010202039C1F800010020C4F80805A5608D
:10D2700025600220C4F80403357070BDF42A002034
:10D2800018040040080000400040024024E000E094
:10D2900070B515460E460446FFF7C0FF31462046DE
:10D2A0002560BDE87040FFF789BF0000017B4FF4A7
:10D2B000803088400149C1F80803704700400240AF
:10D2C0000870020A4A70020C8A70000EC8700420AE
:10D2D0007047000010B50248FDF711FA002010BD9C
:10D2E0007C2B002010B514210448FBF7AFF804484C
:10D2F0000068FDF7BDF9002010BD0000C8500020F7
:10D3000004D8070030B50F2490F8553000220BB137
:10D31000042B03D190F86450012D06D0DD0707D00F
:10D3200090F85650012D02D002E0826E0DE0826D21
:10D330009B070AD590F85C30012B06D1064B006E96
:10D34000C3F5FC23984205D802440AB101240A60BF
:10D35000204630BD0424FBE70080070030B10068A0
:10D360000549884205D048F20250704748F2015002
:10D3700070470020704700006E52464870B5FEF7B7
:10D38000E1FC002811D00020084A094B094C01217A
:10D39000166801FA00F52E4203D004EB8005C5F8AB
:10D3A0000036401CC0B20728F2D370BD080501400A
:10D3B0003546526E00000140FFF7E0BF0020704785
:10D3C000002070472DE9FC4180461C4617460E465A
:10D3D0000C48089DFDF796F910B11120BDE8FC81BD
:10D3E000A20839463046FEF7DDFA0648FDF787F910
:10D3F00033463A4601214046CDE90045FCF7BCFFE3
:10D400000020EBE77C2B00202DE9F84F114D8846DA
:10D4100081461E4617466946DDF828A02868FDF7B4
:10D4200042F9040013D01C21FBF710F800202071F2
:10D43000C4F80090C4E90486C4E902A769462868D4
:10D44000FDF752F9FFF730FB0020BDE8F88F04200C
:10D45000FBE7000004D80700FB37984B72C1537BF1
:10D4600086FBA6698C90BC63E61CBC46941E3C01FE
:10D470009C20B0130112EE2C426F19BDBBDC973516
:10D48000C5CB0DD445D7211CA3C566FD9552621F9F
:10D49000B0B786B83E09F22B0D0E0F100B0C181901
:10D4A0000338FDD87047000039BD07003FBD0700B5
:10D4B00015BD0700200000007800000000000000FB
:10D4C0004800280000204000958707000000000069
:10D4D0000100010000000000010000000000000049
:10D4E0000200050001000000220000000000000012
:10D4F000000000000000000000000000000000002C
:10D500000100010000000000010000000000000018
:10D5100002000500010000004200000000000000C1
:10D5200000000000000000000000000000000000FB
:10D53000010011000400FCFF0400000000000000D6
:10D54000020011000400FCFF0400000000000000C5
:10D55000030021000400FCFF040010000000000094
:10D56000040011000100FFFF0100000000000000A6
:10D57000050011000200FEFF040000000000000092
:10D58000060011000400FCFF040000000000000081
:10D59000070011000400FCFF040000000000000070
:10D5A000080017000200FEFF24000000D0D407008E
:10D5B000090010000100FFFF01000000CCD40700AB
:10D5C0000A0027000200FEFF4400030000D5070008
:10D5D000000000000000000000000000000000004B
:10D5E000010011000100FFFF010000000000000029
:10D5F000020017000200FEFF6401000030D50700A2
:10D60000000000000000000000000000000000001A
:10D61000010007000000000068010000E0D50700DD
:10D6200002000100000000000100000000000000F6
:10D63000030005000100000042000000000000009F
:10D6400000000000000000000000000000000000DA
:10D65000010017000400FCFF68010000E0D507008E
:10D66000020017000400FCFFAC01000010D6070008
:10D6700000000000000000000000000000000000AA
:10D68000001103000011130002000000010000005F
:10D690000338FDD870470C000C0000005802000051
:10D6A0000200000000000000020000000000000076
:10D6B000C42F00200900000000000000000000004E
:10D6C0000100000000000000280000000000000031
:10D6D0000000000000010000000001000000000048
:10D6E000000000000000000000000000000000003A
:10D6F000359A070000000000000000000000000054
:10D700000200000000000100000000000000000016
:10D710000800000000000000359A07007DBF0700E8
:10D7200000000000000000000400000000000000F5
:10D7300000000000000000000000000000000000E9
:10D7400000000000000000000000000000000000D9
:10D75000F4000000000000001800000000000000BD
:10D7600000000000000000000000000000000000B9
:10D7700000000000000000000000000000000000A9
:10D78000170000000000000050EADA308883B89FDC
:10D79000604F15F30000C98E020000000000000079
:10D7A0000000000000000000040000000000000075
:10D7B0000000000000000000000000000000000069
:10D7C0000001000000000000000000000000000058
:10D7D0000000000000000000001000000400000035
:10D7E000010000004DA50700D5D20700CDCA0700F3
:10D7F000C5D30700E5A20700A1CB0700BDD30700F2
:10D8000091A50700DC4E002000100000040000007D
:10D810000100000059A50700E5D20700DBCA070098
:10D8200009D407002DA30700A5CB0700C1D307002B
:10D83000A1A50700982F8A4291443771CFFBC0B54C
:10D84000A5DBB5E95BC25639F111F159A4823F92CB
:10D85000D55E1CAB98AA07D8015B8312BE85312424
:10D86000C37D0C55745DBE72FEB1DE80A706DC9BE5
:10D8700074F19BC1C1699BE48647BEEFC69DC10F91
:10D88000CCA10C246F2CE92DAA84744ADCA9B05CCD
:10D89000DA88F97652513E986DC631A8C82703B090
:10D8A000C77F59BFF30BE0C64791A7D55163CA069E
:10D8B00067292914850AB72738211B2EFC6D2C4DAA
:10D8C000130D385354730A65BB0A6A762EC9C28198
:10D8D000852C7292A1E8BFA24B661AA8708B4BC22E
:10D8E000A3516CC719E892D1240699D685350EF458
:10D8F00070A06A1016C1A419086C371E4C7748270F
:10D90000B5BCB034B30C1C394AAAD84E4FCA9C5B84
:10D91000F36F2E68EE828F746F63A5781478C884D5
:10D920000802C78CFAFFBE90EB6C50A4F7A3F9BEB7
:10D93000F27871C6F0DA0700F8DA0700000000009C
:10D94000000000000100000734D9070044D9070097
:10D95000080000006CD907007CD90700080000000F
:10D960007CD907008CD907000800000010DB0700F5
:10D9700018DB0700000000000000000000DB0700CB
:10D9800010DB0700000000000000000000000000A5
:10D99000000000000000000000000000E8DA0700BE
:10D9A000F0DA07000000000000000000E82A002074
:10D9B0008CD90700ACD9070008000000F8DA07008E
:10D9C00000DB07000000000000000000BCD90700D9
:10D9D000CCD90700080000008DC1070035C1070041
:10D9E000DDC0070053C0070059C0070011C0070081
:10D9F0005FC007009DC00700000000000820000174
:10DA0000FFFFFFFFFFFFFFFFFFFFFFFF0000000022
:10DA1000000000000000000001000000FFFFFFFF09
:10DA2000512563FCC2CAB9F3849E17A7ADFAE6BCC0
:10DA3000FFFFFFFFFFFFFFFF00000000FFFFFFFFF2
:10DA400096C298D84539A1F4A033EB2D817D037798
:10DA5000F240A463E5E6BCF847422CE1F2D1176B33
:10DA6000F551BF376840B6CBCE5E316B5733CE2B06
:10DA7000169E0F7C4AEBE78E9B7F1AFEE242E34F35
:10DA80004B60D2273E3CCE3BF6B053CCB0061D6572
:10DA9000BC86987655BDEBB3E7933AAAD835C65AFB
:10DAA00043860700C9930700E591070024DB0700C0
:10DAB000E82A0020BC00000044960700E0DB0700D5
:10DAC000A42B00203C2D0000549607004D9B07001E
:10DAD000ED9A07003C2B0020143000202530002058
:10DAE00028300020F4000000E59B07000000000043
:10DAF0009DB7070000000000D5B707000000000038
:10DB0000B9BA0700000000002DBC070000000000AB
:10DB1000B5B707000000000000000000030000008F
:10DB2000C9B0070000000000000000000000000075
:10DB300000000000042B0020142B00200000000037
:10DB400000000000000000000000000000000000D5
:10DB500000000000000000000000000001000000C4
:10DB60000000000000000000FF00FFFF00000000B8
:10DB700000000000000000000000000000000000A5
:10DB80000000000001000000000000000000000094
:10DB90000000000000E0070000000000000000009E
:10DBA0000000000000000000000000000000000075
:10DBB0000000000000000000000000000000000065
:10DBC00000000000000000000090D00300000000F2
:10DBD0000000000005A2070000100000000008007F
:10E00000D6C2C4D9020000000100000001000000D7
:10E010000000000000000000300F0100C44E6AB98B
:10E0200001000000000000000000000000000000EF
:10E0300000000000000000000000000000000000E0
:10E0400000000000000000000000000000000000D0
:10E0500000000000000000000000000000000000C0
:10E0600000000000000000000000000000000000B0
:10E250000000000000000000000000008FD41084C7
:10E2600000000000000000000000000000000000AE
:10E27000000000000000000000000000000000009E
:10E28000000000000000000000000000000000008E
:10E29000000000000000000000000000000000007E
:10E2A0000001C44E6AB90000000000000000000038
:10E2B000000000000000000000000000000000005E
:10E2C000000000000000000000000000000000004E
:10E2D000000000000000000000000000000000003E
:10E2E000000000000000000000000000000000002E
:10E2F000000000000000000000000000000000001E
:10E30000000000000000000000000000000000000D
:10E3100000000000000000000000000000000000FD
:04E32000000000FFFA
:10F00000D6C2C4D9020000000100000001000000C7
:10F010000000000000000000300F0100C44E6AB97B
:10F0200001000000000000000000000000000000DF
:10F0300000000000000000000000000000000000D0
:10F0400000000000000000000000000000000000C0
:10F0500000000000000000000000000000000000B0
:10F0600000000000000000000000000000000000A0
:10F250000000000000000000000000008FD41084B7
:10F26000000000000000000000000000000000009E
:10F27000000000000000000000000000000000008E
:10F28000000000000000000000000000000000007E
:10F29000000000000000000000000000000000006E
:10F2A0000001C44E6AB90000000000000000000028
:10F2B000000000000000000000000000000000004E
:10F2C000000000000000000000000000000000003E
:10F2D000000000000000000000000000000000002E
:10F2E000000000000000000000000000000000001E
:10F2F000000000000000000000000000000000000E
:10F3000000000000000000000000000000000000FD
:10F3100000000000000000000000000000000000ED
:04F32000000000FFEA
:020000041000EA
:081014000080070000E0070066
:00000001FF
